:10000000A203040000000000000000000000000047
:1000100000000000000000000000000000000000E0
:1000200000000000000000000000000000000000D0
:1000300000000000000000000000000000000000C0
:1000400000000000000000000000000000000000B0
:1000500000000000000000000000000000000000A0
:100060000000000000000000000000000000000090
:100070000000000000000000000000000000000080
:100080000000000000000000000000000000000070
:100090000000000000000000000000000000000060
:1000A0000000000000000000000000000000000050
:1000B0000000000000000000000000000000000040
:1000C0000000000000000000000000000000000030
:1000D0000000000000000000000000000000000020
:1000E0000000000000000000000000000000000010
:1000F0000000000000000000000000000000000000
:1001000000000000000000000000000000000000EF
:1001100000000000000000000000000000000000DF
:1001200000000000000000000000000000000000CF
:1001300000000000000000000000000000000000BF
:1001400000000000000000000000000000000000AF
:10015000000000000000000000000000000000009F
:10016000000000000000000000000000000000008F
:10017000000000000000000000000000000000007F
:10018000000000000000000000000000000000006F
:10019000000000000000000000000000000000005F
:1001A000000000000000000000000000000000004F
:1001B000000000000000000000000000000000003F
:1001C000000000000000000000000000000000002F
:1001D000000000000000000000000000000000001F
:1001E000000000000000000000000000000000000F
:1001F00000000000000000000000000000000000FF
:100744008F802000F0FF200020A0B70000002000D0
:1007540034A0B700400020004420B7004004020049
:10076400000000008A1F78008B1F7800F0FF2F0024
:10077400A8A2B700C602A900C622A900D262A90095
:100784003B0020004A2D2000DEFF07009EFF0700EB
:1007940064FF0700AB0F2000DA15200046FF0700B6
:1007A4004B1F2000FA19200043FF0700EB1520001F
:1007B400DA15200040FF0700DB0720008A1B200019
:1007C4003DFF07004B1F2000BA2020003AFF07001E
:1007D4007B1720008A1B200037FF0700DB0720005F
:1007E400BA20200034FF0700AB2820003A2920005B
:1007F40031FF07004A1F2000D6FE070049FF07000B
:10080400AB0F2000DA1520002BFF07004B1F200040
:10081400FA19200028FF07007B172000DA152000B2
:1008240025FF0700DB072000BA20200022FF070075
:100834004B1F20008A1B20001FFF07007B1720008E
:10084400DA1520001CFF0700DB072000BA20200077
:1008540019FF0700AB2820008A1B200016FF0700A1
:10086400AA282000BBFE0700C8FF3700CF05780088
:080874004F057800FFFF37007B
:100708000000FA001A408800100020000B00DD00ED
:100718003040880000A0EE00204088001A0D6000DC
:100728001040800062015000920078004080200054
:0C073800108960000080FA00000006003C
:10060C008A1F78008B1F78004B1F20008A1B20004C
:10061C00A7FF07004B1F20008A1B2000A4FF070028
:10062C004B1F20008A1B2000A1FF0700EB152000A8
:10063C00DA1520009EFF07006B092000BA2020006D
:10064C009BFF07004B1F20008A1B200098FF070010
:10065C00EB152000DA15200095FF07006B09200030
:10066C00BA20200092FF0700AB2820008A1B200034
:10067C008FFF07004A1F200034FF07004B1F20008C
:10068C003A2920008AFF07004B1F20003A2920003E
:10069C0087FF07004B1F20003A29200084FF07002A
:1006AC00EB152000AA2B200081FF07006B0920000E
:1006BC00BA2020007EFF07004B1F2000FA192000F3
:1006CC007BFF0700EB152000DA15200078FF0700F0
:1006DC006B092000BA20200075FF0700AB28200012
:1006EC008A1B200072FF07004A1F200017FF07001B
:0C06FC00CF0578004F05780000000600D4
:1004BC008A1F78008B1F7800AEFF0700CF057800ED
:1004CC000040800022002000110009000200D8002A
:1004DC00010078006000E10005003A00CA02A800A3
:1004EC000B05780099FF0700CA02A9000400370029
:1004FC00CA22A8000B05780094FF0700CA22A900A5
:10050C002A03200091FF070011002000008020002A
:0C051C00108840004F0578000000060029
:100380001000FA00F2FF070010079800B3FF070003
:10039000823E200003002000B3FF07008B1F78007F
:1003A0000A0178008001EB000002EB00BFFF0700AC
:1003B0001E0190008001EB000002EB00BBFF070074
:1003C000CF0578008100D1000080D300000798009D
:1003D000A2FF07000B0178008001EB00A2FF0700DD
:1003E00060079800710798001E0090004101DD0031
:1003F0000E0090008000EB008001EB009AFF0700E8
:1004000020079800310798006E009000FE009000D1
:100410002E019000BE0190000002EB00A3FF070038
:10042000800178000102780012072000E0004700F8
:1004300060004700110811006018E10060A0E100B1
:100440001700360010408000100178006180200005
:1004500010408000110871008A9FBE000E059000B8
:100460008005EB0066FF0700104080001001780057
:100470004180200010408000110861000E059000AE
:100480008005EB005EFF07004F05BE006180510054
:10049000E0005A008001780001027800E6FF370092
:1004A0001040800010017800418020001040800042
:0C04B000110861000080FA000000060046
:0803500040002000000006003F
:0C025C0000A02F000100200000000600A0
:100200000A0478004001200000A0EC00900478006F
:100210001000F800E70020008703E9000300350024
:100220008904D1000884D300FBFF37001200F900D5
:10023000F7FF2300878464001000E200040032000E
:10024000F93F0900000000000804E900FAFF370048
:0C0250000980090000000000000006000A
:100268000000FA00020AB800500088000200B80036
:1002780081004200032AB800810042000080FA0091
:04028800000006006C
:1002AC000000FA0002000700A40104000000000096
:1002BC000800E20002003A001000070000000600EF
:1002CC00839F68000200E20002003D006000100005
:1002DC00E08018000600E20002003D006001110001
:1002EC00E0811900050007004F00E00002003B0010
:1002FC0060001000E0801800000006006022B800CA
:10030C00060220000000D0008180D2000482D200BE
:10031C008582D2000000A8000202520083825A009B
:10032C0003003B000202420083824A000000A1004D
:10033C000603E900F3FF3A00000006000080FA0013
:04034C0000000600A7
:100358006050E100070032008A1F78008A3E2000C2
:10036800C8FF07004F0578006100550000057800B8
:08037800F7FF3700000006004A
:10028C006050E1000500320000000000000000009A
:10029C006100550000057800F9FF370000000600EA
:0002AC0052
:100528008A1F78008B1F78004B1F20000A37200095
:10053800E0FF0700CB1220008A1B2000DDFF070028
:100548006B0920008A1B2000DAFF07004B1F2000E0
:100558000A372000D7FF07005B142000EA33200089
:10056800D4FF0700FB0A20000A312000D1FF070052
:10057800DB0720004A2E2000CEFF0700DB07200003
:10058800AA2B2000CBFF0700AB0F20004A2E20002B
:10059800C8FF07005A1420006DFF0700AB0F2000AA
:1005A8007A1C2000C3FF07004B1F2000EA2620000A
:1005B800C0FF07005B142000BA242000BDFF07001D
:1005C800FB0A2000AA222000BAFF0700DB07200050
:1005D800BA202000B7FF0700DB0720002A1D2000F3
:1005E800B4FF0700AB0F2000BA202000B1FF0700BE
:1005F800EA15200056FF0700CF0578004F05780060
:0406080000000600E8
:1008800001802000E043280000000900B018780033
:04089000000006005E
:04087C000000000078
:0200000401F009
:1C000000068300003F000000B38700000F3100000F3300000700000003C0000096
:00000001FF
